
 Start  Stop   Length Name                   Class
 00000H 00003H 00004H CODE                   CODE
 00010H 01EB2H 01EA3H CODE_FAR               CODE
 01EB4H 03C7BH 01DC8H _TEXT                  CODE
 03C80H 0480FH 00B90H CODE                   CODE
 04810H 04B0BH 002FCH CODE                   CODE
 04B10H 04B9FH 00090H CODE                   CODE
 04BA0H 04BF2H 00053H CODE                   CODE
 04C00H 05DCEH 011CFH CODE                   CODE
 05DD0H 06833H 00A64H CODE                   CODE
 06840H 06C57H 00418H CODE                   CODE
 06C60H 06DB3H 00154H CODE                   CODE
 06DC0H 06F09H 0014AH CODE                   CODE
 06F10H 06F38H 00029H CODE                   CODE
 06F40H 06F73H 00034H CODE                   CODE
 06F80H 070A9H 0012AH CODE                   CODE
 070B0H 07178H 000C9H CODE                   CODE
 07180H 072D8H 00159H CODE                   CODE
 072E0H 07465H 00186H CODE                   CODE
 07470H 074BBH 0004CH CODE                   CODE
 074C0H 075EEH 0012FH CODE                   CODE
 075F0H 07802H 00213H CODE                   CODE
 07810H 07B17H 00308H CODE                   CODE
 07B20H 07D29H 0020AH CODE                   CODE
 07D30H 07F5EH 0022FH CODE                   CODE
 07F60H 0814CH 001EDH CODE                   CODE
 08150H 081C1H 00072H CODE                   CODE
 081C2H 081C2H 00000H C_ETEXT                ENDCODE
 081C2H 0C14DH 03F8CH DATA                   DATA
 0C150H 0C2CAH 0017BH DATA                   DATA
 0C2D0H 14F25H 08C56H SELECT                 SELECT
 14F30H 151A5H 00276H SERVICE                SERVICE
 151B0H 159AFH 00800H OUR_STACK              
 159B0H 161CAH 0081BH PARSER                 PARSER
 161D0H 161D0H 00000H PCINPUT                PCINPUT
 161D0H 18B13H 02944H PCINPUT                PCINPUT
 18B20H 18B20H 00000H ZSEG                   ZSEG
 18B20H 18B61H 00042H NULL                   BEGDATA
 18B62H 19079H 00518H _DATA                  DATA
 1907AH 19087H 0000EH CDATA                  DATA
 19088H 19088H 00000H XIFB                   DATA
 19088H 19088H 00000H XIF                    DATA
 19088H 19088H 00000H XIFE                   DATA
 19088H 19088H 00000H XIB                    DATA
 19088H 19088H 00000H XI                     DATA
 19088H 19088H 00000H XIE                    DATA
 19088H 19088H 00000H XPB                    DATA
 19088H 19088H 00000H XP                     DATA
 19088H 19088H 00000H XPE                    DATA
 19088H 19088H 00000H XCB                    DATA
 19088H 19088H 00000H XC                     DATA
 19088H 19088H 00000H XCE                    DATA
 19088H 19088H 00000H XCFB                   DATA
 19088H 19088H 00000H XCF                    DATA
 19088H 19088H 00000H XCFE                   DATA
 19088H 19088H 00000H CONST                  CONST
 19088H 1908FH 00008H HDR                    MSG
 19090H 1915DH 000CEH MSG                    MSG
 1915EH 1915FH 00002H PAD                    MSG
 19160H 19160H 00001H EPAD                   MSG
 19162H 19162H 00000H _BSS                   BSS
 19162H 19162H 00000H XOB                    BSS
 19162H 19162H 00000H XO                     BSS
 19162H 19162H 00000H XOE                    BSS
 19170H 19DB9H 00C4AH c_common               BSS
 19DC0H 1A5BFH 00800H STACK                  STACK

 Origin   Group
 0000:0   AGROUP
 18B2:0   DGROUP

  Address         Publics by Name

 0000:CB82       $M_CLS_1
 0000:CF0F       $M_CLS_2
 0000:C4B1       $M_GET_MSG_ADDRESS
 0000:CF34       $M_MSGSERV_1
 0000:CF55       $M_MSGSERV_2
 0000:8DFF       $M_RT
 0000:C393       ABORT_SELECT
 0000:8502       ACTIVE
 0000:4BD7       ADD_REFRESH
 0000:4F11       ADJUST_DOWN
 0000:4EFC       ADJUST_UP
 0000:50E6       ALLOCATE_BLOCK
 0000:5080       ALLOCATE_HELP
 0000:5148       ALLOCATE_LVB
 0000:5020       ALLOCATE_MEMORY_CALL
 0000:8503       ALTERNATE
 0000:0001  Abs  ALT_FRENCH
 0000:0002  Abs  ALT_FR_ITEMS
 0000:9689       ALT_ID_DEF
 0000:0002  Abs  ALT_ITALIAN
 0000:0002  Abs  ALT_IT_ITEMS
 0000:9674       ALT_KYBD_FR
 0000:9675       ALT_KYBD_FR_1
 0000:967B       ALT_KYBD_IT
 0000:967C       ALT_KYBD_IT_1
 0000:9682       ALT_KYBD_UK
 0000:9683       ALT_KYBD_UK_1
 0000:9662       ALT_KYB_ID
 0000:9663       ALT_KYB_ID_PREV
 0000:0003  Abs  ALT_KYB_ITEMS
 0000:9664       ALT_KYB_TABLE
 0000:9665       ALT_KYB_TAB_1
 0000:9660       ALT_TAB_PTR
 0000:0003  Abs  ALT_UK
 0000:0002  Abs  ALT_UK_ITEMS
 0000:0620       APPEND_STRING_ROUTINE
 18B2:0042       asm2cInRegs
 18B2:0050       asm2coutregs
 18B2:005E       asm2csegregs
 0000:CF76       BCHAR
 0000:077B       BEEP_ROUTINE
 0000:07A2       BIN_TO_CHAR_ROUTINE
 0000:0002       BOXDR
 0000:0002  Abs  CGA
 0000:0233       CHANGE_ATTRIBUTE_ROUTINE
 0000:1D24       CHANGE_AUTOEXEC_ROUTINE
 0000:04D8       CHECK_DISK_ROUTINE
 0000:0010       CHECK_DOS_PATH_ROUTINE
 0000:BAC8       CHECK_FILE
 0000:4B5E       CHECK_MIN_MAX
 0000:052B       CHECK_VALID_MEDIA_ROUTINE
 0000:0068       CHECK_VALID_PATH
 0000:CF77       CHECK_VERSION
 0000:02C2       CHECK_WRITE_ROUTINE
 0000:0ABA       CHK_EX_MEM_ROUTINE
 0000:8209       CHK_W_PROTECT_FLAG
 0000:041E       CHMOD_FILE_ROUTINE
 0000:E430       choose_shell_screen
 0000:4B49       CLEAR_USER_STRING
 0000:03CB       CLOSE_FILE_ROUTINE
 0000:9A32       CMD_BUFF
 06F1:0000       COLOR
 0000:0298       COMPARE_ROUTINE
 075F:0000       COMPE
 0000:0690       CONTINUE_360
 0000:4B71       CONVERT_ASCII
 0000:4BA6       CONVERT_NUMERIC
 0000:8607       COPY_INST_1200_1440
 0000:87CD       COPY_OPER_1200_1440
 0000:0644       COPY_ROUTINE
 0000:85E3       COPY_SEL_EGA
 0000:85EF       COPY_SEL_LCD
 0000:85FB       COPY_SEL_SHEL
 0000:8911       COPY_SHELL_1200_1440
 0000:A701       CRD_CCBVECOFF
 0000:A703       CRD_CCBVECSEG
 0000:1F50       CREATE_AUTOEXEC_BAT
 0000:263E       CREATE_CONFIG_SYS
 0000:03E0       CREATE_FILE_ROUTINE
 0000:2CFA       CREATE_SHELL_BAT
 0815:0000       CRITE
 0000:000C  Abs  CTY_A_ITEMS
 0000:000B  Abs  CTY_B_ITEMS
 0000:94CD       CTY_TAB_A
 0000:94CE       CTY_TAB_A_1
 0000:9582       CTY_TAB_B
 0000:9583       CTY_TAB_B_1
 0000:3741       CURSOROFF
 0000:3755       CURSORON
 07D3:0000       DATES
 0000:F760       DATE_TIME_SCREEN
 0000:5125       DEALLOCATE_BLOCK
 0000:50C3       DEALLOCATE_HELP
 0000:5183       DEALLOCATE_LVB
 0000:5068       DEALLOCATE_MEMORY_CALL
 0000:BAC6       DEST_PANEL
 0000:0E20       DISKETTE_INSTALL
 0000:9D4C       DISK_1_START
 0000:9D4A       DISK_1_TABLE
 0000:9D4B       DISK_1_VAL_ITEM
 0000:A136       DISK_2_START
 0000:A134       DISK_2_TABLE
 0000:A135       DISK_2_VAL_ITEM
 0000:A5A1       DISK_PANEL
 0000:0CE9       DISPLAY_MESSAGE_ROUTINE
 0000:4919       DISPLAY_PANEL_CALL
 03C8:0000       DISPQ
 07B2:008A       DISP_MODEG
 0000:DDE0       DOS_LOC_SCREEN
 0000:E7C0       DOS_PARAMETERS_SCREEN
 0000:0000  Abs  DRIVE_A
 0000:0001  Abs  DRIVE_B
 0000:8501       DSKCPY_ERR
 0000:84F8       DSKCPY_OPTION
 0000:84FB       DSKCPY_PAN1
 0000:84FD       DSKCPY_PAN2
 0000:84FF       DSKCPY_PAN3
 0000:84F9       DSKCPY_SOURCE
 0000:84F7       DSKCPY_WHICH
 0000:8FC8       D_ANSI_1
 0000:9087       D_BUFFERS_1
 0000:908B       D_BUFFERS_2
 0000:947D       D_DOS_LOC_1
 0000:90E6       D_FASTOPEN_1
 0000:90F2       D_FASTOPEN_2
 0000:910B       D_FCBS_1
 0000:911F       D_FILES_1
 0000:9123       D_FILES_2
 0000:9184       D_LASTDRIVE_1
 0000:9280       D_PROMPT_1
 0000:9310       D_SHELL_1
 0000:9332       D_SHELL_2
 0000:9412       D_XMA2EMS_1
 0000:0003  Abs  EGA
 0000:03FF       ERASE_FILE_ROUTINE
 0000:45CF       ERROR_ACTIVE
 0000:8FAD       ERROR_KEYS
 0000:0003  Abs  ERROR_KEYS_LEN
 0000:84EA       EXEC_DEALLOC
 0000:84E7       EXEC_ERR
 0000:84EB       EXEC_FDISK
 0000:0898       EXEC_PROGRAM_ROUTINE
 0000:478E       EXEC_SCROLL_CALL
 0000:1EB3       EXIT_DOS
 0000:1EC9       EXIT_DOS_CONT
 0000:C2F1       EXIT_SELECT
 0000:C372       EXIT_SELECT2
 0000:0002  Abs  E_ANSI_B
 0000:0003  Abs  E_ANSI_C
 0000:0002  Abs  E_ANSI_NO
 0000:0001  Abs  E_ANSI_YES
 0000:0002  Abs  E_APPEND_NO
 0000:0001  Abs  E_APPEND_YES
 0000:0000  Abs  E_CLEAN_NO
 0000:0001  Abs  E_CLEAN_YES
 0000:0001  Abs  E_CPSW_B
 0000:0001  Abs  E_CPSW_C
 0000:0000  Abs  E_CPSW_DISP
 0000:0006  Abs  E_CPSW_NA
 0000:0002  Abs  E_CPSW_NO
 0000:0001  Abs  E_CPSW_NOT_REC
 0000:0000  Abs  E_CPSW_NOT_VAL
 0000:0002  Abs  E_CPSW_VALID
 0000:0001  Abs  E_CPSW_YES
 0000:000D  Abs  E_CR
 0000:0001  Abs  E_CTY_KB_PREDEF
 0000:0002  Abs  E_CTY_KB_USER
 0000:0001  Abs  E_CTY_LIST_1
 0000:0002  Abs  E_CTY_LIST_2
 0000:0001  Abs  E_DEST_DOS
 0000:0003  Abs  E_DEST_DRIVE_A
 0000:0002  Abs  E_DEST_DRIVE_B
 0000:0001  Abs  E_DEST_DRIVE_C
 0000:0000  Abs  E_DEST_SELECT
 0000:0002  Abs  E_DEST_SHELL
 0000:0001  Abs  E_DEST_USER
 0000:0001  Abs  E_DISK1_INSTALL
 0000:0002  Abs  E_DISK1_REPLACE
 0000:0001  Abs  E_DISKETTE_1200
 0000:0007  Abs  E_DISKETTE_1440
 0000:0000  Abs  E_DISKETTE_360
 0000:0002  Abs  E_DISKETTE_720
 0000:00FF  Abs  E_DISKETTE_INV
 0000:0001  Abs  E_DISK_1
 0000:0002  Abs  E_DISK_2
 0000:0013  Abs  E_DISK_COL
 0000:0008  Abs  E_DISK_EDOS_MEM
 0000:0002  Abs  E_DISK_EXT_DOS
 0000:0010  Abs  E_DISK_FREE_MEM
 0000:0000  Abs  E_DISK_INV
 0000:0004  Abs  E_DISK_LOG_DRI
 0000:0001  Abs  E_DISK_NO_PART
 0000:0001  Abs  E_DISK_PRI
 0000:0000  Abs  E_DISK_ROW
 0000:0002  Abs  E_DISK_VAL_PART
 0000:0013  Abs  E_DRIVE_COL
 0000:0000  Abs  E_DRIVE_ROW
 0000:0000  Abs  E_DSKCPY_OK
 0000:0001  Abs  E_DSKCPY_RETRY
 0000:000D  Abs  E_ENTER
 0000:0001  Abs  E_ENTIRE_DISK
 0000:001B  Abs  E_ESCAPE
 0000:3D00  Abs  E_F3
 0000:0004  Abs  E_FASTOPEN_C
 0000:0002  Abs  E_FASTOPEN_NO
 0000:0001  Abs  E_FASTOPEN_YES
 0000:0002  Abs  E_FILES
 0000:0000  Abs  E_FILE_ATTR
 0000:0001  Abs  E_FORMAT_FAT
 0000:0002  Abs  E_FORMAT_NEW
 0000:0002  Abs  E_FORMAT_NO
 0000:0001  Abs  E_FORMAT_SELECT
 0000:0003  Abs  E_FORMAT_USED
 0000:0005  Abs  E_FREE_MEM_DISK
 0000:0004  Abs  E_FREE_MEM_EDOS
 0000:0003  Abs  E_GRAFTABL_B
 0000:0005  Abs  E_GRAFTABL_C
 0000:0006  Abs  E_GRAFTABL_NA
 0000:0002  Abs  E_GRAFTABL_NO
 0000:0001  Abs  E_GRAFTABL_YES
 0000:0004  Abs  E_GRAPHICS_B
 0000:0006  Abs  E_GRAPHICS_C
 0000:0002  Abs  E_GRAPHICS_NO
 0000:0001  Abs  E_GRAPHICS_YES
 0000:0006  Abs  E_HIDE_SEL
 0000:0005  Abs  E_HIDE_STARTUP
 0000:0019  Abs  E_INST_1200_1440
 0000:0001  Abs  E_IS_MOD80
 0000:0000  Abs  E_KYBD_ALT_NO
 0000:0001  Abs  E_KYBD_ALT_YES
 0000:0001  Abs  E_KYBD_LIST_1
 0000:0002  Abs  E_KYBD_LIST_2
 0000:0002  Abs  E_KYBD_VAL_DEF
 0000:0000  Abs  E_KYBD_VAL_NO
 0000:0001  Abs  E_KYBD_VAL_YES
 0000:0002  Abs  E_KYB_LOAD_ERR
 0000:0001  Abs  E_KYB_LOAD_SUC
 0000:0004  Abs  E_KYB_LOAD_UND
 0000:0003  Abs  E_KYB_LOAD_US
 0000:000A  Abs  E_LF
 0000:0006  Abs  E_NA
 0000:0002  Abs  E_NO
 0000:0001  Abs  E_NOCPSW_DISP
 0000:0000  Abs  E_NOT_MOD80
 0000:001B  Abs  E_OPER_1200_1440
 0000:0002  Abs  E_OPTION_A_C
 0000:0001  Abs  E_OPTION_B_C
 0000:0050  Abs  E_PARALLEL
 0000:0001  Abs  E_PART_DEFAULT
 0000:0002  Abs  E_PART_EXT_DOS
 0000:0001  Abs  E_PART_FAT
 0000:0001  Abs  E_PART_FORMAT
 0000:0004  Abs  E_PART_IGNORE
 0000:0002  Abs  E_PART_KSAM
 0000:0003  Abs  E_PART_LOG_DRI
 0000:0006  Abs  E_PART_OTHER
 0000:0001  Abs  E_PART_PRI_DOS
 0000:0003  Abs  E_PART_UNDEF
 0000:0000  Abs  E_PART_UNFORMAT
 0000:0002  Abs  E_PART_USER
 0000:0002  Abs  E_PATH_NO
 0000:0002  Abs  E_PATH_ONLY
 0000:0001  Abs  E_PATH_YES
 0000:0002  Abs  E_PROMPT_NO
 0000:0001  Abs  E_PROMPT_YES
 0000:0001  Abs  E_QUIT
 0000:0002  Abs  E_RETURN
 0000:0001  Abs  E_REVIEW_ACCEPT
 0000:0002  Abs  E_REVIEW_VIEW
 0000:0001  Abs  E_SELECT_FDISK
 0000:00FF  Abs  E_SELECT_INV
 0000:0000  Abs  E_SELECT_MENU
 0000:0001  Abs  E_SEL_EGA
 0000:0001  Abs  E_SEL_LCD
 0000:0001  Abs  E_SEL_SHEL
 0000:0053  Abs  E_SERIAL
 0000:0007  Abs  E_SHARE_C
 0000:0002  Abs  E_SHARE_NO
 0000:0001  Abs  E_SHARE_YES
 0000:0006  Abs  E_SHELL_1200_1440
 0000:0005  Abs  E_SHELL_B
 0000:0008  Abs  E_SHELL_C
 0000:0002  Abs  E_SHELL_NO
 0000:0001  Abs  E_SHELL_YES
 0000:0020  Abs  E_SPACE
 0000:0002  Abs  E_SPACE_DISK
 0000:0001  Abs  E_SPACE_EDOS
 0000:0000  Abs  E_SPACE_NONE
 0000:0009  Abs  E_TAB
 0000:0006  Abs  E_VDISK_B
 0000:0009  Abs  E_VDISK_C
 0000:0002  Abs  E_VDISK_NO
 0000:0001  Abs  E_VDISK_YES
 0000:0002  Abs  E_WORKSPACE_BAL
 0000:0003  Abs  E_WORKSPACE_MAX
 0000:0001  Abs  E_WORKSPACE_MIN
 0000:0000  Abs  E_XMA_ABSENT
 0000:0002  Abs  E_XMA_C
 0000:0006  Abs  E_XMA_NA
 0000:0002  Abs  E_XMA_NO
 0000:0001  Abs  E_XMA_PRESENT
 0000:0001  Abs  E_XMA_YES
 0000:0001  Abs  E_YES
 0000:0441       FIND_FILE_ROUTINE
 0000:F09D       FIRST_DISK_SCREEN
 0000:8FA5       FK_DATE
 0000:0004  Abs  FK_DATE_LEN
 0000:8F8A       FK_ENT
 0000:8F84       FK_ENT_ESC
 0000:8F86       FK_ENT_ESC_F3
 0000:0004  Abs  FK_ENT_ESC_F3_LEN
 0000:0002  Abs  FK_ENT_ESC_LEN
 0000:8F81       FK_ENT_F3
 0000:0003  Abs  FK_ENT_F3_LEN
 0000:0001  Abs  FK_ENT_LEN
 0000:8FA9       FK_FORMAT
 0000:0003  Abs  FK_FORMAT_LEN
 0000:8FAC       FK_REBOOT
 0000:0000  Abs  FK_REBOOT_LEN
 0000:8F9E       FK_REVIEW
 0000:0007  Abs  FK_REVIEW_LEN
 0000:8F91       FK_SCROLL
 0000:0006  Abs  FK_SCROLL_LEN
 0000:8F97       FK_TAB
 0000:0007  Abs  FK_TAB_LEN
 0000:8F8B       FK_TEXT
 0000:0006  Abs  FK_TEXT_LEN
 0781:0000       FMTFD
 0000:FBB0       FORMAT_DISK_SCREEN
 0000:A5A0       FORMAT_WHICH
 0000:1F3A       Free_Parser
 0000:8FCC       F_ANSI
 0000:9072       F_APPEND
 0000:909F       F_CPSW
 0000:9100       F_FASTOPEN
 0000:9D46       F_FORMAT
 0000:917F       F_GRAFTABL
 0000:917D       F_GRAPHICS
 0000:9D42       F_PARTITION
 0000:9204       F_PATH
 0000:9286       F_PROMPT
 0000:9A15       F_REVIEW
 0000:9299       F_SHARE
 0000:9388       F_SHELL
 0000:93B2       F_VDISK
 0000:9432       F_XMA
 06F8:0000       GEQUP
 0000:09BC       GET_CNTY_DEF_ROUTINE
 0000:0A17       GET_CNTY_INDEX_ROUTINE
 0000:F744       GET_ENTER_KEY
 0000:492F       GET_FUNCTION_CALL
 0000:4E46       GET_HELP_ID
 0000:3608       GET_ICB
 0000:2EAE       GET_INPUT_CALL
 0000:2F3D       GET_KEY
 0000:0A51       GET_KYBD_INDEX_ROUTINE
 0000:0A94       GET_KYBD_ROUTINE
 0000:0DCD       GET_OVERLAY
 0000:35B6       GET_PCB
 0000:1A75       GET_PRINTER_INFO_ROUTINE
 0000:0B5D       GET_PRINTER_PARAMS_ROUTINE
 0000:174F       GET_PRINTER_TITLES_ROUTINE
 0000:35DF       GET_SCB
 0000:2DF0       GET_SCROLL_CALL
 0000:4957       GET_STRING_CALL
 01EB:001E       gget_status
 0000:0003       GRAPH
 0481:0000       GVIDO
 0000:4710       HANDLE_CHILDREN
 0000:45D0       HANDLE_ERROR_CALL
 0000:4501       HANDLE_F3
 0000:46FD       HANDLE_KEYSTROKE
 0000:46B5       HANDLE_PANEL_CALL
 0000:46D6       HANDLE_PANEL_CALL2
 0000:46F6       HANDLE_PANEL_CALL3
 0000:8733       HIDE_SEL
 0000:8787       HIDE_STARTUP
 0684:000E       HLPRD
 0000:0CFF       HOOK_INT_23
 0000:0D3D       HOOK_INT_24
 0000:0D93       HOOK_INT_2F
 0000:0DCB       HOOK_INT_2F_256KB
 0000:0DF0       HOOK_INT_2F_FORMAT
 0000:A635       HRD_BUFLEN
 0000:A637       HRD_BUFOFF
 0000:A639       HRD_BUFSEG
 070B:0000       IN2ST
 06C6:0000       INCHA
 0000:A6D3       INC_KS
 0000:0001       INDBC
 0000:CF5F       INITIALIZATION
 0000:38BF       INITIALIZE
 0000:4C2F       INIT_CHAR_CALL
 0000:4750       INIT_PQUEUE_CALL
 0000:47FD       INIT_SCROLL_CALL
 0000:4AF1       INIT_SCROLL_STATUS_CALL
 0000:4859       INIT_SCROLL_W_LIST_CALL
 0000:488A       INIT_SCROLL_W_NUM_CALL
 0000:49F0       INIT_STRING_CALL
 161D:1988       INPUT
 0000:3B6D       INSERT_DISK_ROUTINE
 0000:C2D4       INSTALL
 0000:1F0A       INSTALL_ERROR
 0000:15D0       INSTALL_TO_360_DRIVE
 04B1:0000       INSTRN
 0000:D56C       INTRO_SCREEN
 0000:15A5       INT_23_VECTOR
 0000:A58F       INT_24_ERROR
 0000:A591       INT_24_FLAG
 0000:0E24       INT_24_VECTOR
 0000:13F6       INT_2F_256KB
 0000:136E       INT_2F_FORMAT
 0000:108F       INT_2F_VECTOR
 0000:A9D4       IN_CCBVECOFF
 0000:A9D6       IN_CCBVECSEG
 0000:A9D8       IN_CURNOR
 0000:A9C8       IN_ICBID
 0000:94B0       I_COUNTRY
 0000:94AC       I_CTY_KYBD
 0000:9D44       I_DESTINATION
 0000:9438       I_DEST_DRIVE
 0000:94B6       I_KEYBOARD
 0000:94C4       I_KYBD_ALT
 0000:99A8       I_PORT
 0000:99AC       I_PRINTER
 0000:99AA       I_REDIRECT
 0000:8EFB       I_USER_INDEX
 0000:8FC0       I_WORKSPACE
 0000:B9B0       KD_BACKSPACE
 0000:0009  Abs  KYBD_A_ITEMS
 0000:0009  Abs  KYBD_B_ITEMS
 0000:9628       KYBD_TAB_A
 0000:9629       KYBD_TAB_A_1
 0000:9644       KYBD_TAB_B
 0000:9645       KYBD_TAB_B_1
 0000:0004  Abs  LCD
 0000:938A       MACHINE_TYPE
 0000:0697       MAKE_DIR_PATHS_ROUTINE
 0000:034F       MATCH_FILES_ROUTINE
 0000:001F  Abs  MAX_DAY
 0000:0017  Abs  MAX_HOUR
 0000:8F01       MAX_INPUT_VAL
 0000:003B  Abs  MAX_MINUTE
 0000:000C  Abs  MAX_MONTH
 0000:855B       MAX_NAME
 0000:0007  Abs  MAX_NUMPRINT
 0000:003B  Abs  MAX_SECOND
 0000:081F  Abs  MAX_YEAR
 04BA:0000       MBEEP
 0000:0080  Abs  MC_LINE
 0000:A59E       MEM_SIZE
 0000:0001  Abs  MIN_DAY
 0000:0000  Abs  MIN_HOUR
 0000:8EFF       MIN_INPUT_VAL
 0000:0000  Abs  MIN_MINUTE
 0000:0001  Abs  MIN_MONTH
 0000:0000  Abs  MIN_NUMPRINT
 0000:0000  Abs  MIN_SECOND
 0000:07BC  Abs  MIN_YEAR
 0000:00FA  Abs  MOD25_OR_MOD30
 0000:3BE0       MOD_XCOPY
 0000:0001  Abs  MONO
 072E:0000       MOVEC
 07B2:0000       MOVEG
 0747:0000       MOVEI
 0718:0000       MOVEM
 0000:0003  Abs  MT_BREAK
 0000:0007  Abs  MT_BUFFERS
 0000:0003  Abs  MT_CPSW
 0000:0007  Abs  MT_FCBS
 0000:0003  Abs  MT_FILES
 0000:0001  Abs  MT_LASTDRIVE
 0000:0006  Abs  MT_STACKS
 0000:0003  Abs  MT_VERIFY
 0000:0002  Abs  M_ANSI
 0000:0078  Abs  M_APPEND
 0000:0028  Abs  M_APPEND_P
 0000:0003  Abs  M_BREAK
 0000:0007  Abs  M_BUFFERS
 0000:0003  Abs  M_CPSW
 0000:0016  Abs  M_CP_DRIVER
 0000:000C  Abs  M_CP_PREPARE
 0000:0003  Abs  M_DEST_DRIVE
 0000:0064  Abs  M_DISK_1_ITEMS
 0000:0064  Abs  M_DISK_2_ITEMS
 0000:0025  Abs  M_DOS_LOC
 0000:003C  Abs  M_FASTOPEN
 0000:0007  Abs  M_FCBS
 0000:0003  Abs  M_FILES
 0000:0050  Abs  M_GRAPHICS
 0000:0014  Abs  M_GRAPH_PARM
 0000:0028  Abs  M_INSTALL_PATH
 0000:0002  Abs  M_KEYBOARD
 0000:0002  Abs  M_KYBD_ALT
 0000:0001  Abs  M_LASTDRIVE
 0000:0028  Abs  M_MODE_PARM
 0000:0078  Abs  M_PATH
 0000:000A  Abs  M_PRINT_FILE
 0000:0078  Abs  M_PROMPT
 0000:000F  Abs  M_SHARE
 0000:0073  Abs  M_SHELL
 0000:0006  Abs  M_STACKS
 0000:0078  Abs  M_STR120_1
 0000:0078  Abs  M_STR120_2
 0000:0078  Abs  M_STR120_3
 0000:0078  Abs  M_STR120_4
 0000:0028  Abs  M_STR40
 0000:0078  Abs  M_USER_STRING
 0000:0014  Abs  M_VDISK
 0000:0003  Abs  M_VERIFY
 0000:0028  Abs  M_XMA2EMS
 0000:0028  Abs  M_XMAEM
 0000:8542       NAMES_OFF
 0000:9D2F       N_BYTE_1
 0000:9D21       N_COUNTER
 0000:94B2       N_COUNTRY
 0000:90A6       N_CPSW
 0000:94BF       N_CP_PRI
 0000:94C1       N_CP_SEC
 0000:94AE       N_CTY_LIST
 0000:94C3       N_CTY_RES
 0000:9A1C       N_DAY
 0000:94BD       N_DESIGNATES
 0000:A58E       N_DEST
 0000:943C       N_DEST_DRIVE
 0000:9D48       N_DISK1_MODE
 0000:943E       N_DISKETTE_A
 0000:943F       N_DISKETTE_B
 0000:943D       N_DISKETTE_TOT
 0000:9D36       N_DISK_1
 0000:9D3A       N_DISK_1_S1
 0000:9D3E       N_DISK_1_S2
 0000:9D38       N_DISK_2
 0000:9D3C       N_DISK_2_S1
 0000:9D40       N_DISK_2_S2
 0000:A528       N_DISK_NUM
 0000:9A17       N_DISPLAY
 0000:943A       N_DRIVE_OPTION
 0000:9D35       N_DSKCPY_ERR
 0000:8FB2       N_FORMAT_MODE
 0000:9D19       N_HANDLE
 0000:9A1E       N_HOUR
 0000:9D34       N_HOUSE_CLEAN
 0000:94CA       N_KYBD_ALT
 0000:94B4       N_KYBD_LIST
 0000:94BC       N_KYBD_VAL
 0000:94CB       N_KYB_LOAD
 0000:A524       N_LEVEL1_PART
 0000:A525       N_LEVEL2_PART
 0000:A526       N_LEVEL3_PART
 0000:A527       N_LEVEL4_PART
 0000:9A20       N_MINUTE
 0000:9436       N_MOD80
 0000:9A1A       N_MONTH
 0000:A51E       N_NAME_PART
 0000:99A2       N_NUMPRINT
 0000:99A4       N_PARALLEL
 0000:99AE       N_PRINTER_TYPE
 0000:8557       N_PRN_NAMES
 0000:9D1F       N_RETCODE
 0000:9A22       N_SECOND
 0000:8FB0       N_SELECT_MODE
 0000:99A6       N_SERIAL
 0000:A51F       N_SIZE_PART
 0000:A521       N_STATUS_PART
 0000:A522       N_TYPE_PART
 0000:8F7F       N_USER_FUNC
 0000:8EFD       N_USER_NUMERIC
 0000:8F7D       N_VALID_KEYS
 0000:9D23       N_WORD_1
 0000:9D25       N_WORD_2
 0000:9D27       N_WORD_3
 0000:9D29       N_WORD_4
 0000:9D2B       N_WORD_5
 0000:9D2D       N_WORD_6
 0000:8FC2       N_WORK_PREV
 0000:9D1D       N_WRITE_ERR_CODE
 0000:9D1B       N_WRITE_HANDLE
 0000:9434       N_XMA
 0000:9A18       N_YEAR
 0000:0000  Abs  N_ZERO_DISKETTE
 0000:A592       OLD_INT_23
 0000:A596       OLD_INT_24
 0000:A59A       OLD_INT_2F
 0000:0460       OPEN_FILE_ROUTINE
 05DD:001E       PANEL
 0000:9A24       PARM_BLOCK
 0000:377F       PCDISPQ_CALL
 0000:389F       PCGVIDO_CALL
 0000:388C       PCINPUT_CALL
 0000:3803       PCMBEEP_CALL
 0000:378F       PCPANEL_CALL
 0000:3813       PCSLCTP_CALL
 0000:A7FA       PM_BASEATTR
 0000:A7F9       PM_BASECHAR
 0000:067B       POP_ROUTINE
 0000:076C       POS_ZERO
 0000:07D8       PREPARE_FILE_ROUTINE
 0000:477C       PREPARE_PANEL_CALL
 0000:DFDB       PRINTER_SCREEN
 0000:9692       PRINTER_TABLES
 0000:1EA4       PROCESS_ESC_F3
 0000:938B       PS2_FLAG
 0000:0664       PUSH_ROUTINE
 0000:A523       P_DRIVE_PART
 0000:9AAF       P_STR120_1
 0000:9A85       P_STR40
 0000:8F05       P_USER_STRING
 0000:A77D       QM_ACTIVEPAN
 0000:A77B       QM_ID
 0000:A777       QM_OPT1
 0000:A779       QM_OPT2
 0000:04AE       READ_FILE_ROUTINE
 0000:1D00       RELEASE_PRINTER_INFO_ROUTINE
 0000:02B6       REMOVE_END_BLANKS
 0000:047F       RENAME_FILE_ROUTINE
 0000:0D28       RESTORE_INT_23
 0000:0D72       RESTORE_INT_24
 0000:0DB8       RESTORE_INT_2F
 0000:4BFF       RETURN_STRING_CALL
 06F4:0000       ROWCL
 0000:9D30       SAVE_AREA
 0000:0857       SAVE_FILE_ROUTINE
 0000:0C34       SAVE_PRINTER_PARAMS_ROUTINE
 0000:0566       SCAN_DISK_TABLE_ROUTINE
 0000:D5A6       SCAN_INFO_CALL
 0000:161C       SCAN_INFO_FILE_ROUTINE
 0000:15B9       SCAN_PARAMETERS_ROUTINE
 0000:8B26       SC_1
 0000:8B2A       SC_2
 0000:82F6       SC_DISPLAY_EGA
 0000:8305       SC_DISPLAY_LCD
 0000:8B36       SC_EXT
 0000:9C95       SC_LINE
 0000:8B3E       SC_LOG
 0000:8B2E       SC_PRI
 0000:8300       SD_DISPLAY_EGA
 0000:830F       SD_DISPLAY_LCD
 0000:A5A3       SEARCH_FILE
 0000:8540       SEG_LOC
 0000:A52A       SELECT_STACK
 0000:853F       SEL_FLG
 0000:1E3C       SET_DISPLAY_MODE_ROUTINE
 0000:48A9       SET_SCROLL_CALL
 0000:489E       SET_SCROLL_COLOUR
 0000:4A60       SET_STRING_CALL
 0000:0001  Abs  SHELL
 0000:0001  Abs  SH_FILES
 0000:002D  Abs  SIZE_NAMES
 04C0:0000       SLCTP
 0000:BAC4       SOURCE_PANEL
 0000:A529       STACK_INDEX
 0000:0064  Abs  STACK_SIZE
 0000:0000  Abs  STARTUP
 18B2:04F0       STKHQQ
 074C:0000       STRST
 0000:9079       ST_BREAK
 0000:9091       ST_BUFFERS
 0000:90A1       ST_CPSW
 0000:9111       ST_FCBS
 0000:9126       ST_FILES
 0000:9187       ST_LASTDRIVE
 0000:9394       ST_STACKS
 0000:93B9       ST_VERIFY
 0000:A5A5       SUB_ERROR
 0000:8EE7       SUPPORT_STATUS
 0000:C5D8       SYSDISPMSG
 0000:5A4F       SYSPARSE
 0000:8FC4       S_ANSI
 0000:8D0F       S_ANSI_B
 0000:8D96       S_ANSI_C
 0000:8FCE       S_APPEND
 0000:8D1D       S_APPEND_B
 0000:8DA2       S_APPEND_C
 0000:9048       S_APPEND_P
 0000:8CDF       S_AUTOEX_C
 0000:8A76       S_AUTO_C
 0000:8ACD       S_AUTO_FDISK
 0000:8AC7       S_AUTO_MENU
 0000:89D3       S_AUTO_NEW
 0000:8A32       S_AUTO_NEW_B
 0000:8A98       S_AUTO_NEW_C
 0000:8AB8       S_AUTO_REBOOT
 0000:8A54       S_AUTO_REN
 0000:944E       S_A_DRIVE
 0000:8BB0       S_A_STARS
 0000:9074       S_BREAK
 0000:907E       S_BUFFERS
 0000:9452       S_B_DRIVE
 0000:8BC7       S_COLON
 0000:89A8       S_COMMAND_COM
 0000:8AD4       S_CONFIG_AUTO
 0000:8A88       S_CONFIG_C
 0000:89E2       S_CONFIG_NEW
 0000:8A44       S_CONFIG_NEW_B
 0000:8AA9       S_CONFIG_NEW_C
 0000:8A66       S_CONFIG_REN
 0000:8CEF       S_CONSYS_C
 0000:909A       S_CPSW
 0000:99D9       S_CP_DRIVER
 0000:99F1       S_CP_PREPARE
 0000:8C23       S_CP_SEL
 0000:944A       S_C_DRIVE
 0000:9440       S_DEST_DRIVE
 0000:8B0F       S_DISKCOPY
 0000:8B1E       S_DISKCOPY_PARM
 0000:899B       S_DOS_COM_360
 0000:9456       S_DOS_LOC
 0000:8966       S_DOS_SEL_360
 0000:8959       S_DOS_SHEL_DISK
 0000:8973       S_DOS_UTIL1_DISK
 0000:8980       S_DOS_UTIL2_DISK
 0000:898E       S_DOS_UTIL3_DISK
 0000:9445       S_DRIVE_A
 0000:8B53       S_DRIVE_C
 0000:8C41       S_DSKCPY_TO_B
 0000:90A8       S_FASTOPEN
 0000:8D74       S_FASTOPEN_B
 0000:8DEF       S_FASTOPEN_C
 0000:9102       S_FCBS
 0000:8B03       S_FDISK
 0000:911A       S_FILES
 0000:8B46       S_FORMAT
 0000:8B71       S_FORMAT_A
 0000:8B57       S_FORMAT_B
 0000:8D2D       S_GRAFTABL_B
 0000:8DB0       S_GRAFTABL_C
 0000:912B       S_GRAPHICS
 0000:8D3F       S_GRAPHICS_B
 0000:8DC0       S_GRAPHICS_C
 0000:8D51       S_GRAPHPRO_B
 0000:8DD0       S_GRAPHPRO_C
 0000:99FF       S_GRAPH_PARM
 0000:9482       S_INSTALL_PATH
 0000:8AF8       S_KEYB
 0000:94B8       S_KEYBOARD
 0000:94C6       S_KYBD_ALT
 0000:9181       S_LASTDRIVE
 0000:8C33       S_MODE
 0000:99AF       S_MODE_PARM
 0000:8FB7       S_OFF
 0000:8FBC       S_ON
 0000:89FF       S_OS2_AUTO_C
 0000:89EF       S_OS2_CONFIG_C
 0000:918A       S_PATH
 0000:8BE9       S_PREP_EGA
 0000:8C06       S_PREP_LCD
 0000:89C6       S_PRINT_FILE
 0000:9206       S_PROMPT
 0000:8D63       S_RECOVER_B
 0000:8DE0       S_RECOVER_C
 0000:8B8B       S_REPLACE
 0000:8B99       S_REPLACE_PAR1
 0000:8CA7       S_SELCOM_C
 0000:8C49       S_SELCOM_NEW_B
 0000:8C99       S_SELDAT_C
 0000:8C89       S_SELDAT_NEW_B
 0000:89B9       S_SELECT_TMP
 0000:8CD1       S_SELEXE_C
 0000:8C79       S_SELEXE_NEW_B
 0000:8CB5       S_SELHLP_C
 0000:8C59       S_SELHLP_NEW_B
 0000:8CC3       S_SELPRT_C
 0000:8C69       S_SELPRT_NEW_B
 0000:9288       S_SHARE
 0000:929B       S_SHELL
 0000:8AEC       S_SHELL2
 0000:8A11       S_SHELL_NEW
 0000:8A20       S_SHELL_NEW_B
 0000:8C3E       S_SLASH
 0000:8BB8       S_SLASH_A
 0000:8BC2       S_SLASH_Q
 0000:8BAB       S_SLASH_R
 0000:8BBD       S_SLASH_S
 0000:8FB4       S_SPACE
 0000:938C       S_STACKS
 0000:9AAD       S_STR120_1
 0000:9B27       S_STR120_2
 0000:9BA1       S_STR120_3
 0000:9C1B       S_STR120_4
 0000:9A83       S_STR40
 0000:968E       S_SWISS
 0000:8BCA       S_SYS_C
 0000:968A       S_US
 0000:8F03       S_USER_STRING
 0000:939C       S_VDISK
 0000:8CFD       S_VDISK_B
 0000:8D86       S_VDISK_C
 0000:93B4       S_VERIFY
 0000:8BD4       S_VOL_SEL
 0000:93E8       S_XMA2EMS
 0000:93BE       S_XMAEM
 07F6:0008       TIMES
 0000:4B05       TOGGLE_SUPPORT_CALL
 0000:4B2C       UNPAD_USER_STRING
 0000:05C8       UPDATE_DISK_TABLE_ROUTINE
 0000:ED60       VDISK_SCREEN
 0000:4F30       VIDEO_CHECK
 0000:D610       WORKSPACE_SCREEN
 0000:04C3       WRITE_FILE_ROUTINE
 0000:0824       WRITE_LINE_ROUTINE
 0000:ACC1       WR_DATA2LEN
 0000:ACBF       WR_DATA2OFF
 0000:ACBD       WR_DATA2SEG
 0000:AC32       WR_DRETLEN
 0000:AC34       WR_DRETOFF
 0000:AC36       WR_DRETSEG
 0000:ACBB       WR_ERROR
 0000:AC48       WR_HCBCONT
 0000:AC3E       WR_HLPOPT
 0000:AC44       WR_HLPROW
 0000:ACEB       WR_ICBVEC
 0000:ACC7       WR_LVBLEN
 0000:ACC9       WR_LVBMEM
 0000:ACC5       WR_LVBOFF
 0000:ACC3       WR_LVBSEG
 0000:ACCF       WR_MAXHELPSZ
 0000:ACCB       WR_MAXMEMPAR
 0000:0014  Abs  WR_MAXREFID
 0000:AC8D       WR_REFBUF
 0000:AC8B       WR_REFCNT
 0000:AC91       WR_REFID
 0000:AC8F       WR_REFIELDCNT
 0000:AC85       WR_REFNUM
 0000:AC87       WR_REFOFF
 0000:AC89       WR_REFSEG
 0000:ACB9       WR_SCBID
 06DC:000C       WWRAP
 0000:820A       W_PROTECT_FLAG
 18B2:0FD0       _boot_record
 01EB:13E6       _copy_fdisk2select
 18B2:11D2       _cur_disk
 18B2:0BD5       _cur_disk_buff
 01EB:1399       _cylinders_to_mbytes
 01EB:1768       _DiskIo
 18B2:0692       _display_page
 18B2:0651       _dx_buff
 18B2:0642       _edata
 18B2:12A0       _end
 18B2:0532       _environ
 18B2:050B       _errno
 18B2:1298       _errorlevel
 01EB:19F2       _exit
 18B2:0BB0       _extended_buff
 18B2:0BBA       _extended_flag
 18B2:0698       _ext_table
 18B2:008C       _fat12_String
 18B2:0090       _fat16_String
 01EB:0B89       _find_ext_free_space
 01EB:135B       _find_logical_drive
 01EB:1285       _find_partition_location
 01EB:1301       _find_partition_system_type
 01EB:12C4       _find_partition_type
 01EB:08DC       _find_part_free_space
 18B2:008A       _format_string
 18B2:11D4       _free_space
 01EB:15B0       _get_disk_info
 01EB:1692       _get_drive_parameters
 01EB:1525       _get_num_logical_dos_drives
 01EB:1571       _get_partition_size
 01EB:00B2       _get_status
 18B2:0696       _good_disk
 18B2:0094       _hilda_string
 01EB:041D       _init_partition_tables
 18B2:067A       _input_col
 18B2:0680       _input_data
 18B2:0694       _input_row
 18B2:0BD6       _insert
 01EB:184E       _int86x
 01EB:0F8D       _load_logical_drive
 18B2:11D0       _logical_buff
 18B2:0BB8       _logical_flag
 0000:0000       _MAIN
 18B2:0098       _master_boot_record
 18B2:0678       _max_head
 18B2:1299       _max_partition_size
 18B2:0FCE       _max_sector
 18B2:0691       _next_letter
 18B2:0086       _NOVAL
 18B2:0BD4       _no_fatal_error
 18B2:0BB9       _number_of_drives
 18B2:066C       _OneDiskStatusEntry
 18B2:0EF6       _part_table
 18B2:0084       _pinsert
 18B2:0BB6       _primary_buff
 18B2:0690       _primary_flag
 01EB:16E8       _read_boot_record
 18B2:0650       _reboot_flag
 18B2:0682       _regs
 18B2:1294       _required_cyls
 18B2:0BA8       _segregs
 18B2:0BBC       _sort
 01EB:0EF9       _sort_ext_table
 01EB:0E47       _sort_part_table
 18B2:0BB2       _total_disk
 18B2:067C       _total_mbytes
 18B2:11D3       _valid_input
 01EB:0118       _valid_stat
 18B2:0676       _video_mode
 18B2:04EE       __abrkp
 18B2:049E       __abrktb
 18B2:04EE       __abrktbe
 18B2:04F2       __acfinfo
 0000:9876  Abs  __acrtmsg
 0000:9876  Abs  __acrtused
 18B2:0542       __adbgmsg
 18B2:049C       __aexit_rtn
 18B2:04FF       __aintdiv
 01EB:1829       __amsg_exit
 01EB:18E2       __aNlmul
 01EB:1916       __aNlshl
 01EB:18E2       __aNulmul
 01EB:1922       __aNulshr
 18B2:0498       __asizds
 01EB:1786       __astart
 18B2:049A       __atopsp
 18B2:053A       __child
 01EB:1838       __chkstk
 01EB:192E       __cinit
 01EB:181A       __cintDIV
 01EB:1A4E       __ctermsub
 18B2:0516       __doserrno
 01EB:1D30       __dosret0
 01EB:1D43       __dosretax
 01EB:1D38       __dosreturn
 18B2:0513       __dosvermajor
 18B2:0514       __dosverminor
 01EB:1A09       __exit
 18B2:0503       __fac
 01EB:1A9E       __FF_MSGBANNER
 18B2:055C       __fpinit
 01EB:1D84       __fptrap
 18B2:053D       __intno
 01EB:1D50       __maperror
 01EB:1D8A       __myalloc
 18B2:0518       __nfile
 01EB:1CDC       __NMSG_TEXT
 01EB:1D07       __NMSG_WRITE
 01EB:1ABE       __nullcheck
 18B2:0516       __oserr
 18B2:051A       __osfile
 18B2:0513       __osmajor
 18B2:0514       __osminor
 18B2:0515       __osmode
 18B2:0513       __osversion
 18B2:053C       __ovlflag
 18B2:053E       __ovlvec
 18B2:0534       __pgmptr
 18B2:0511       __psp
 18B2:050F       __pspadr
 01EB:1AE0       __setargv
 01EB:1C6E       __setenvp
 18B2:050D       __umaskval
 18B2:052E       ___argc
 18B2:0530       ___argv

  Address         Publics by Value

 0000:0000  Abs  E_DRIVE_ROW
 0000:0000  Abs  E_DISKETTE_360
 0000:0000  Abs  E_DEST_SELECT
 0000:0000  Abs  MIN_MINUTE
 0000:0000  Abs  MIN_NUMPRINT
 0000:0000  Abs  E_DISK_INV
 0000:0000  Abs  N_ZERO_DISKETTE
 0000:0000  Abs  E_SELECT_MENU
 0000:0000  Abs  STARTUP
 0000:0000  Abs  MIN_SECOND
 0000:0000  Abs  E_FILE_ATTR
 0000:0000  Abs  E_KYBD_ALT_NO
 0000:0000  Abs  E_SPACE_NONE
 0000:0000  Abs  E_XMA_ABSENT
 0000:0000  Abs  E_DISK_ROW
 0000:0000  Abs  E_NOT_MOD80
 0000:0000  Abs  E_PART_UNFORMAT
 0000:0000  Abs  E_CPSW_DISP
 0000:0000  Abs  E_CLEAN_NO
 0000:0000  Abs  FK_REBOOT_LEN
 0000:0000  Abs  DRIVE_A
 0000:0000       _MAIN
 0000:0000  Abs  E_KYBD_VAL_NO
 0000:0000  Abs  E_DSKCPY_OK
 0000:0000  Abs  MIN_HOUR
 0000:0000  Abs  E_CPSW_NOT_VAL
 0000:0001  Abs  SHELL
 0000:0001  Abs  E_CTY_LIST_1
 0000:0001  Abs  E_KYBD_ALT_YES
 0000:0001  Abs  E_PART_PRI_DOS
 0000:0001  Abs  E_DISK1_INSTALL
 0000:0001  Abs  E_WORKSPACE_MIN
 0000:0001  Abs  E_VDISK_YES
 0000:0001  Abs  E_CPSW_NOT_REC
 0000:0001  Abs  E_SEL_EGA
 0000:0001  Abs  E_SEL_SHEL
 0000:0001  Abs  E_CTY_KB_PREDEF
 0000:0001  Abs  E_SHELL_YES
 0000:0001  Abs  E_IS_MOD80
 0000:0001  Abs  SH_FILES
 0000:0001  Abs  E_ENTIRE_DISK
 0000:0001  Abs  E_XMA_YES
 0000:0001  Abs  MONO
 0000:0001  Abs  E_SELECT_FDISK
 0000:0001  Abs  E_KYBD_LIST_1
 0000:0001  Abs  E_GRAPHICS_YES
 0000:0001  Abs  E_PART_FORMAT
 0000:0001  Abs  E_DSKCPY_RETRY
 0000:0001  Abs  MT_LASTDRIVE
 0000:0001  Abs  E_SHARE_YES
 0000:0001  Abs  E_PROMPT_YES
 0000:0001  Abs  E_OPTION_B_C
 0000:0001  Abs  E_DISKETTE_1200
 0000:0001  Abs  E_PATH_YES
 0000:0001  Abs  E_DEST_USER
 0000:0001  Abs  MIN_DAY
 0000:0001  Abs  E_FASTOPEN_YES
 0000:0001  Abs  E_REVIEW_ACCEPT
 0000:0001  Abs  E_DEST_DRIVE_C
 0000:0001  Abs  E_PART_DEFAULT
 0000:0001  Abs  E_FORMAT_FAT
 0000:0001  Abs  E_CPSW_C
 0000:0001  Abs  E_APPEND_YES
 0000:0001  Abs  E_KYBD_VAL_YES
 0000:0001  Abs  E_CPSW_B
 0000:0001  Abs  FK_ENT_LEN
 0000:0001  Abs  E_NOCPSW_DISP
 0000:0001  Abs  E_DEST_DOS
 0000:0001  Abs  DRIVE_B
 0000:0001  Abs  E_YES
 0000:0001       INDBC
 0000:0001  Abs  E_SEL_LCD
 0000:0001  Abs  ALT_FRENCH
 0000:0001  Abs  E_KYB_LOAD_SUC
 0000:0001  Abs  E_FORMAT_SELECT
 0000:0001  Abs  E_DISK_PRI
 0000:0001  Abs  E_ANSI_YES
 0000:0001  Abs  E_CPSW_YES
 0000:0001  Abs  E_DISK_1
 0000:0001  Abs  E_XMA_PRESENT
 0000:0001  Abs  E_DISK_NO_PART
 0000:0001  Abs  E_QUIT
 0000:0001  Abs  E_CLEAN_YES
 0000:0001  Abs  E_GRAFTABL_YES
 0000:0001  Abs  M_LASTDRIVE
 0000:0001  Abs  E_PART_FAT
 0000:0001  Abs  E_SPACE_EDOS
 0000:0001  Abs  MIN_MONTH
 0000:0002  Abs  M_KEYBOARD
 0000:0002  Abs  E_FORMAT_NEW
 0000:0002  Abs  E_DISK_2
 0000:0002  Abs  E_ANSI_NO
 0000:0002  Abs  E_DISK_EXT_DOS
 0000:0002  Abs  E_PATH_ONLY
 0000:0002  Abs  E_DISKETTE_720
 0000:0002  Abs  M_ANSI
 0000:0002  Abs  E_PART_USER
 0000:0002  Abs  M_KYBD_ALT
 0000:0002  Abs  ALT_FR_ITEMS
 0000:0002  Abs  E_DISK_VAL_PART
 0000:0002  Abs  ALT_UK_ITEMS
 0000:0002  Abs  E_CPSW_NO
 0000:0002  Abs  E_OPTION_A_C
 0000:0002  Abs  E_VDISK_NO
 0000:0002  Abs  E_REVIEW_VIEW
 0000:0002  Abs  E_PROMPT_NO
 0000:0002  Abs  ALT_IT_ITEMS
 0000:0002  Abs  E_PATH_NO
 0000:0002  Abs  E_ANSI_B
 0000:0002  Abs  E_CTY_KB_USER
 0000:0002  Abs  E_DISK1_REPLACE
 0000:0002  Abs  E_PART_EXT_DOS
 0000:0002  Abs  E_XMA_C
 0000:0002  Abs  E_NO
 0000:0002       BOXDR
 0000:0002  Abs  FK_ENT_ESC_LEN
 0000:0002  Abs  E_DEST_DRIVE_B
 0000:0002  Abs  E_CTY_LIST_2
 0000:0002  Abs  E_FILES
 0000:0002  Abs  E_KYB_LOAD_ERR
 0000:0002  Abs  E_GRAFTABL_NO
 0000:0002  Abs  E_DEST_SHELL
 0000:0002  Abs  E_CPSW_VALID
 0000:0002  Abs  E_KYBD_VAL_DEF
 0000:0002  Abs  E_SPACE_DISK
 0000:0002  Abs  E_XMA_NO
 0000:0002  Abs  E_SHARE_NO
 0000:0002  Abs  E_PART_KSAM
 0000:0002  Abs  E_WORKSPACE_BAL
 0000:0002  Abs  E_GRAPHICS_NO
 0000:0002  Abs  E_FASTOPEN_NO
 0000:0002  Abs  E_APPEND_NO
 0000:0002  Abs  CGA
 0000:0002  Abs  E_KYBD_LIST_2
 0000:0002  Abs  E_RETURN
 0000:0002  Abs  ALT_ITALIAN
 0000:0002  Abs  E_SHELL_NO
 0000:0002  Abs  E_FORMAT_NO
 0000:0003  Abs  MT_FILES
 0000:0003  Abs  MT_CPSW
 0000:0003  Abs  E_PART_LOG_DRI
 0000:0003  Abs  M_DEST_DRIVE
 0000:0003  Abs  E_GRAFTABL_B
 0000:0003  Abs  FK_FORMAT_LEN
 0000:0003  Abs  ALT_UK
 0000:0003  Abs  EGA
 0000:0003  Abs  ERROR_KEYS_LEN
 0000:0003  Abs  E_KYB_LOAD_US
 0000:0003  Abs  E_WORKSPACE_MAX
 0000:0003  Abs  FK_ENT_F3_LEN
 0000:0003       GRAPH
 0000:0003  Abs  M_BREAK
 0000:0003  Abs  E_FORMAT_USED
 0000:0003  Abs  E_ANSI_C
 0000:0003  Abs  MT_BREAK
 0000:0003  Abs  E_PART_UNDEF
 0000:0003  Abs  ALT_KYB_ITEMS
 0000:0003  Abs  E_DEST_DRIVE_A
 0000:0003  Abs  MT_VERIFY
 0000:0003  Abs  M_VERIFY
 0000:0003  Abs  M_CPSW
 0000:0003  Abs  M_FILES
 0000:0004  Abs  E_PART_IGNORE
 0000:0004  Abs  FK_ENT_ESC_F3_LEN
 0000:0004  Abs  LCD
 0000:0004  Abs  E_FASTOPEN_C
 0000:0004  Abs  FK_DATE_LEN
 0000:0004  Abs  E_FREE_MEM_EDOS
 0000:0004  Abs  E_GRAPHICS_B
 0000:0004  Abs  E_KYB_LOAD_UND
 0000:0004  Abs  E_DISK_LOG_DRI
 0000:0005  Abs  E_SHELL_B
 0000:0005  Abs  E_HIDE_STARTUP
 0000:0005  Abs  E_GRAFTABL_C
 0000:0005  Abs  E_FREE_MEM_DISK
 0000:0006  Abs  E_HIDE_SEL
 0000:0006  Abs  M_STACKS
 0000:0006  Abs  FK_TEXT_LEN
 0000:0006  Abs  MT_STACKS
 0000:0006  Abs  E_GRAPHICS_C
 0000:0006  Abs  E_SHELL_1200_1440
 0000:0006  Abs  E_GRAFTABL_NA
 0000:0006  Abs  E_PART_OTHER
 0000:0006  Abs  E_VDISK_B
 0000:0006  Abs  E_XMA_NA
 0000:0006  Abs  FK_SCROLL_LEN
 0000:0006  Abs  E_CPSW_NA
 0000:0006  Abs  E_NA
 0000:0007  Abs  FK_TAB_LEN
 0000:0007  Abs  E_SHARE_C
 0000:0007  Abs  M_FCBS
 0000:0007  Abs  FK_REVIEW_LEN
 0000:0007  Abs  M_BUFFERS
 0000:0007  Abs  MT_FCBS
 0000:0007  Abs  MAX_NUMPRINT
 0000:0007  Abs  E_DISKETTE_1440
 0000:0007  Abs  MT_BUFFERS
 0000:0008  Abs  E_DISK_EDOS_MEM
 0000:0008  Abs  E_SHELL_C
 0000:0009  Abs  KYBD_B_ITEMS
 0000:0009  Abs  E_VDISK_C
 0000:0009  Abs  KYBD_A_ITEMS
 0000:0009  Abs  E_TAB
 0000:000A  Abs  E_LF
 0000:000A  Abs  M_PRINT_FILE
 0000:000B  Abs  CTY_B_ITEMS
 0000:000C  Abs  CTY_A_ITEMS
 0000:000C  Abs  M_CP_PREPARE
 0000:000C  Abs  MAX_MONTH
 0000:000D  Abs  E_CR
 0000:000D  Abs  E_ENTER
 0000:000F  Abs  M_SHARE
 0000:0010  Abs  E_DISK_FREE_MEM
 0000:0010       CHECK_DOS_PATH_ROUTINE
 0000:0013  Abs  E_DISK_COL
 0000:0013  Abs  E_DRIVE_COL
 0000:0014  Abs  M_GRAPH_PARM
 0000:0014  Abs  M_VDISK
 0000:0014  Abs  WR_MAXREFID
 0000:0016  Abs  M_CP_DRIVER
 0000:0017  Abs  MAX_HOUR
 0000:0019  Abs  E_INST_1200_1440
 0000:001B  Abs  E_ESCAPE
 0000:001B  Abs  E_OPER_1200_1440
 0000:001F  Abs  MAX_DAY
 0000:0020  Abs  E_SPACE
 0000:0025  Abs  M_DOS_LOC
 0000:0028  Abs  M_APPEND_P
 0000:0028  Abs  M_STR40
 0000:0028  Abs  M_MODE_PARM
 0000:0028  Abs  M_INSTALL_PATH
 0000:0028  Abs  M_XMA2EMS
 0000:0028  Abs  M_XMAEM
 0000:002D  Abs  SIZE_NAMES
 0000:003B  Abs  MAX_MINUTE
 0000:003B  Abs  MAX_SECOND
 0000:003C  Abs  M_FASTOPEN
 0000:0050  Abs  M_GRAPHICS
 0000:0050  Abs  E_PARALLEL
 0000:0053  Abs  E_SERIAL
 0000:0064  Abs  STACK_SIZE
 0000:0064  Abs  M_DISK_2_ITEMS
 0000:0064  Abs  M_DISK_1_ITEMS
 0000:0068       CHECK_VALID_PATH
 0000:0073  Abs  M_SHELL
 0000:0078  Abs  M_STR120_3
 0000:0078  Abs  M_STR120_1
 0000:0078  Abs  M_PROMPT
 0000:0078  Abs  M_USER_STRING
 0000:0078  Abs  M_STR120_4
 0000:0078  Abs  M_APPEND
 0000:0078  Abs  M_STR120_2
 0000:0078  Abs  M_PATH
 0000:0080  Abs  MC_LINE
 0000:00FA  Abs  MOD25_OR_MOD30
 0000:00FF  Abs  E_DISKETTE_INV
 0000:00FF  Abs  E_SELECT_INV
 0000:0233       CHANGE_ATTRIBUTE_ROUTINE
 0000:0298       COMPARE_ROUTINE
 0000:02B6       REMOVE_END_BLANKS
 0000:02C2       CHECK_WRITE_ROUTINE
 0000:034F       MATCH_FILES_ROUTINE
 0000:03CB       CLOSE_FILE_ROUTINE
 0000:03E0       CREATE_FILE_ROUTINE
 0000:03FF       ERASE_FILE_ROUTINE
 0000:041E       CHMOD_FILE_ROUTINE
 0000:0441       FIND_FILE_ROUTINE
 0000:0460       OPEN_FILE_ROUTINE
 0000:047F       RENAME_FILE_ROUTINE
 0000:04AE       READ_FILE_ROUTINE
 0000:04C3       WRITE_FILE_ROUTINE
 0000:04D8       CHECK_DISK_ROUTINE
 0000:052B       CHECK_VALID_MEDIA_ROUTINE
 0000:0566       SCAN_DISK_TABLE_ROUTINE
 0000:05C8       UPDATE_DISK_TABLE_ROUTINE
 0000:0620       APPEND_STRING_ROUTINE
 0000:0644       COPY_ROUTINE
 0000:0664       PUSH_ROUTINE
 0000:067B       POP_ROUTINE
 0000:0697       MAKE_DIR_PATHS_ROUTINE
 0000:076C       POS_ZERO
 0000:077B       BEEP_ROUTINE
 0000:07A2       BIN_TO_CHAR_ROUTINE
 0000:07BC  Abs  MIN_YEAR
 0000:07D8       PREPARE_FILE_ROUTINE
 0000:081F  Abs  MAX_YEAR
 0000:0824       WRITE_LINE_ROUTINE
 0000:0857       SAVE_FILE_ROUTINE
 0000:0898       EXEC_PROGRAM_ROUTINE
 0000:09BC       GET_CNTY_DEF_ROUTINE
 0000:0A17       GET_CNTY_INDEX_ROUTINE
 0000:0A51       GET_KYBD_INDEX_ROUTINE
 0000:0A94       GET_KYBD_ROUTINE
 0000:0ABA       CHK_EX_MEM_ROUTINE
 0000:0B5D       GET_PRINTER_PARAMS_ROUTINE
 0000:0C34       SAVE_PRINTER_PARAMS_ROUTINE
 0000:0CE9       DISPLAY_MESSAGE_ROUTINE
 0000:0CFF       HOOK_INT_23
 0000:0D28       RESTORE_INT_23
 0000:0D3D       HOOK_INT_24
 0000:0D72       RESTORE_INT_24
 0000:0D93       HOOK_INT_2F
 0000:0DB8       RESTORE_INT_2F
 0000:0DCB       HOOK_INT_2F_256KB
 0000:0DF0       HOOK_INT_2F_FORMAT
 0000:0E24       INT_24_VECTOR
 0000:108F       INT_2F_VECTOR
 0000:136E       INT_2F_FORMAT
 0000:13F6       INT_2F_256KB
 0000:15A5       INT_23_VECTOR
 0000:15B9       SCAN_PARAMETERS_ROUTINE
 0000:161C       SCAN_INFO_FILE_ROUTINE
 0000:174F       GET_PRINTER_TITLES_ROUTINE
 0000:1A75       GET_PRINTER_INFO_ROUTINE
 0000:1D00       RELEASE_PRINTER_INFO_ROUTINE
 0000:1D24       CHANGE_AUTOEXEC_ROUTINE
 0000:1E3C       SET_DISPLAY_MODE_ROUTINE
 01EB:001E       gget_status
 01EB:00B2       _get_status
 01EB:0118       _valid_stat
 01EB:041D       _init_partition_tables
 01EB:08DC       _find_part_free_space
 01EB:0B89       _find_ext_free_space
 01EB:0E47       _sort_part_table
 01EB:0EF9       _sort_ext_table
 01EB:0F8D       _load_logical_drive
 01EB:1285       _find_partition_location
 01EB:12C4       _find_partition_type
 01EB:1301       _find_partition_system_type
 01EB:135B       _find_logical_drive
 01EB:1399       _cylinders_to_mbytes
 01EB:13E6       _copy_fdisk2select
 01EB:1525       _get_num_logical_dos_drives
 01EB:1571       _get_partition_size
 01EB:15B0       _get_disk_info
 01EB:1692       _get_drive_parameters
 01EB:16E8       _read_boot_record
 01EB:1768       _DiskIo
 01EB:1786       __astart
 01EB:181A       __cintDIV
 01EB:1829       __amsg_exit
 01EB:1838       __chkstk
 01EB:184E       _int86x
 01EB:18E2       __aNulmul
 01EB:18E2       __aNlmul
 01EB:1916       __aNlshl
 01EB:1922       __aNulshr
 01EB:192E       __cinit
 01EB:19F2       _exit
 01EB:1A09       __exit
 01EB:1A4E       __ctermsub
 01EB:1A9E       __FF_MSGBANNER
 01EB:1ABE       __nullcheck
 01EB:1AE0       __setargv
 01EB:1C6E       __setenvp
 01EB:1CDC       __NMSG_TEXT
 01EB:1D07       __NMSG_WRITE
 01EB:1D30       __dosret0
 01EB:1D38       __dosreturn
 01EB:1D43       __dosretax
 01EB:1D50       __maperror
 01EB:1D84       __fptrap
 01EB:1D8A       __myalloc
 03C8:0000       DISPQ
 0000:3D00  Abs  E_F3
 0481:0000       GVIDO
 04B1:0000       INSTRN
 04BA:0000       MBEEP
 04C0:0000       SLCTP
 05DD:001E       PANEL
 0684:000E       HLPRD
 06C6:0000       INCHA
 06DC:000C       WWRAP
 06F1:0000       COLOR
 06F4:0000       ROWCL
 06F8:0000       GEQUP
 070B:0000       IN2ST
 0718:0000       MOVEM
 072E:0000       MOVEC
 0747:0000       MOVEI
 074C:0000       STRST
 075F:0000       COMPE
 0781:0000       FMTFD
 07B2:0000       MOVEG
 07B2:008A       DISP_MODEG
 07D3:0000       DATES
 07F6:0008       TIMES
 0815:0000       CRITE
 0000:8209       CHK_W_PROTECT_FLAG
 0000:820A       W_PROTECT_FLAG
 0000:82F6       SC_DISPLAY_EGA
 0000:8300       SD_DISPLAY_EGA
 0000:8305       SC_DISPLAY_LCD
 0000:830F       SD_DISPLAY_LCD
 0000:84E7       EXEC_ERR
 0000:84EA       EXEC_DEALLOC
 0000:84EB       EXEC_FDISK
 0000:84F7       DSKCPY_WHICH
 0000:84F8       DSKCPY_OPTION
 0000:84F9       DSKCPY_SOURCE
 0000:84FB       DSKCPY_PAN1
 0000:84FD       DSKCPY_PAN2
 0000:84FF       DSKCPY_PAN3
 0000:8501       DSKCPY_ERR
 0000:8502       ACTIVE
 0000:8503       ALTERNATE
 0000:853F       SEL_FLG
 0000:8540       SEG_LOC
 0000:8542       NAMES_OFF
 0000:8557       N_PRN_NAMES
 0000:855B       MAX_NAME
 0000:85E3       COPY_SEL_EGA
 0000:85EF       COPY_SEL_LCD
 0000:85FB       COPY_SEL_SHEL
 0000:8607       COPY_INST_1200_1440
 0000:8733       HIDE_SEL
 0000:8787       HIDE_STARTUP
 0000:87CD       COPY_OPER_1200_1440
 0000:8911       COPY_SHELL_1200_1440
 0000:8959       S_DOS_SHEL_DISK
 0000:8966       S_DOS_SEL_360
 0000:8973       S_DOS_UTIL1_DISK
 0000:8980       S_DOS_UTIL2_DISK
 0000:898E       S_DOS_UTIL3_DISK
 0000:899B       S_DOS_COM_360
 0000:89A8       S_COMMAND_COM
 0000:89B9       S_SELECT_TMP
 0000:89C6       S_PRINT_FILE
 0000:89D3       S_AUTO_NEW
 0000:89E2       S_CONFIG_NEW
 0000:89EF       S_OS2_CONFIG_C
 0000:89FF       S_OS2_AUTO_C
 0000:8A11       S_SHELL_NEW
 0000:8A20       S_SHELL_NEW_B
 0000:8A32       S_AUTO_NEW_B
 0000:8A44       S_CONFIG_NEW_B
 0000:8A54       S_AUTO_REN
 0000:8A66       S_CONFIG_REN
 0000:8A76       S_AUTO_C
 0000:8A88       S_CONFIG_C
 0000:8A98       S_AUTO_NEW_C
 0000:8AA9       S_CONFIG_NEW_C
 0000:8AB8       S_AUTO_REBOOT
 0000:8AC7       S_AUTO_MENU
 0000:8ACD       S_AUTO_FDISK
 0000:8AD4       S_CONFIG_AUTO
 0000:8AEC       S_SHELL2
 0000:8AF8       S_KEYB
 0000:8B03       S_FDISK
 0000:8B0F       S_DISKCOPY
 0000:8B1E       S_DISKCOPY_PARM
 0000:8B26       SC_1
 0000:8B2A       SC_2
 0000:8B2E       SC_PRI
 0000:8B36       SC_EXT
 0000:8B3E       SC_LOG
 0000:8B46       S_FORMAT
 0000:8B53       S_DRIVE_C
 0000:8B57       S_FORMAT_B
 0000:8B71       S_FORMAT_A
 0000:8B8B       S_REPLACE
 0000:8B99       S_REPLACE_PAR1
 0000:8BAB       S_SLASH_R
 0000:8BB0       S_A_STARS
 0000:8BB8       S_SLASH_A
 0000:8BBD       S_SLASH_S
 0000:8BC2       S_SLASH_Q
 0000:8BC7       S_COLON
 0000:8BCA       S_SYS_C
 0000:8BD4       S_VOL_SEL
 0000:8BE9       S_PREP_EGA
 0000:8C06       S_PREP_LCD
 0000:8C23       S_CP_SEL
 0000:8C33       S_MODE
 0000:8C3E       S_SLASH
 0000:8C41       S_DSKCPY_TO_B
 0000:8C49       S_SELCOM_NEW_B
 0000:8C59       S_SELHLP_NEW_B
 0000:8C69       S_SELPRT_NEW_B
 0000:8C79       S_SELEXE_NEW_B
 0000:8C89       S_SELDAT_NEW_B
 0000:8C99       S_SELDAT_C
 0000:8CA7       S_SELCOM_C
 0000:8CB5       S_SELHLP_C
 0000:8CC3       S_SELPRT_C
 0000:8CD1       S_SELEXE_C
 0000:8CDF       S_AUTOEX_C
 0000:8CEF       S_CONSYS_C
 0000:8CFD       S_VDISK_B
 0000:8D0F       S_ANSI_B
 0000:8D1D       S_APPEND_B
 0000:8D2D       S_GRAFTABL_B
 0000:8D3F       S_GRAPHICS_B
 0000:8D51       S_GRAPHPRO_B
 0000:8D63       S_RECOVER_B
 0000:8D74       S_FASTOPEN_B
 0000:8D86       S_VDISK_C
 0000:8D96       S_ANSI_C
 0000:8DA2       S_APPEND_C
 0000:8DB0       S_GRAFTABL_C
 0000:8DC0       S_GRAPHICS_C
 0000:8DD0       S_GRAPHPRO_C
 0000:8DE0       S_RECOVER_C
 0000:8DEF       S_FASTOPEN_C
 0000:8DFF       $M_RT
 0000:8EE7       SUPPORT_STATUS
 0000:8EFB       I_USER_INDEX
 0000:8EFD       N_USER_NUMERIC
 0000:8EFF       MIN_INPUT_VAL
 0000:8F01       MAX_INPUT_VAL
 0000:8F03       S_USER_STRING
 0000:8F05       P_USER_STRING
 0000:8F7D       N_VALID_KEYS
 0000:8F7F       N_USER_FUNC
 0000:8F81       FK_ENT_F3
 0000:8F84       FK_ENT_ESC
 0000:8F86       FK_ENT_ESC_F3
 0000:8F8A       FK_ENT
 0000:8F8B       FK_TEXT
 0000:8F91       FK_SCROLL
 0000:8F97       FK_TAB
 0000:8F9E       FK_REVIEW
 0000:8FA5       FK_DATE
 0000:8FA9       FK_FORMAT
 0000:8FAC       FK_REBOOT
 0000:8FAD       ERROR_KEYS
 0000:8FB0       N_SELECT_MODE
 0000:8FB2       N_FORMAT_MODE
 0000:8FB4       S_SPACE
 0000:8FB7       S_OFF
 0000:8FBC       S_ON
 0000:8FC0       I_WORKSPACE
 0000:8FC2       N_WORK_PREV
 0000:8FC4       S_ANSI
 0000:8FC8       D_ANSI_1
 0000:8FCC       F_ANSI
 0000:8FCE       S_APPEND
 0000:9048       S_APPEND_P
 0000:9072       F_APPEND
 0000:9074       S_BREAK
 0000:9079       ST_BREAK
 0000:907E       S_BUFFERS
 0000:9087       D_BUFFERS_1
 0000:908B       D_BUFFERS_2
 0000:9091       ST_BUFFERS
 0000:909A       S_CPSW
 0000:909F       F_CPSW
 0000:90A1       ST_CPSW
 0000:90A6       N_CPSW
 0000:90A8       S_FASTOPEN
 0000:90E6       D_FASTOPEN_1
 0000:90F2       D_FASTOPEN_2
 0000:9100       F_FASTOPEN
 0000:9102       S_FCBS
 0000:910B       D_FCBS_1
 0000:9111       ST_FCBS
 0000:911A       S_FILES
 0000:911F       D_FILES_1
 0000:9123       D_FILES_2
 0000:9126       ST_FILES
 0000:912B       S_GRAPHICS
 0000:917D       F_GRAPHICS
 0000:917F       F_GRAFTABL
 0000:9181       S_LASTDRIVE
 0000:9184       D_LASTDRIVE_1
 0000:9187       ST_LASTDRIVE
 0000:918A       S_PATH
 0000:9204       F_PATH
 0000:9206       S_PROMPT
 0000:9280       D_PROMPT_1
 0000:9286       F_PROMPT
 0000:9288       S_SHARE
 0000:9299       F_SHARE
 0000:929B       S_SHELL
 0000:9310       D_SHELL_1
 0000:9332       D_SHELL_2
 0000:9388       F_SHELL
 0000:938A       MACHINE_TYPE
 0000:938B       PS2_FLAG
 0000:938C       S_STACKS
 0000:9394       ST_STACKS
 0000:939C       S_VDISK
 0000:93B2       F_VDISK
 0000:93B4       S_VERIFY
 0000:93B9       ST_VERIFY
 0000:93BE       S_XMAEM
 0000:93E8       S_XMA2EMS
 0000:9412       D_XMA2EMS_1
 0000:9432       F_XMA
 0000:9434       N_XMA
 0000:9436       N_MOD80
 0000:9438       I_DEST_DRIVE
 0000:943A       N_DRIVE_OPTION
 0000:943C       N_DEST_DRIVE
 0000:943D       N_DISKETTE_TOT
 0000:943E       N_DISKETTE_A
 0000:943F       N_DISKETTE_B
 0000:9440       S_DEST_DRIVE
 0000:9445       S_DRIVE_A
 0000:944A       S_C_DRIVE
 0000:944E       S_A_DRIVE
 0000:9452       S_B_DRIVE
 0000:9456       S_DOS_LOC
 0000:947D       D_DOS_LOC_1
 0000:9482       S_INSTALL_PATH
 0000:94AC       I_CTY_KYBD
 0000:94AE       N_CTY_LIST
 0000:94B0       I_COUNTRY
 0000:94B2       N_COUNTRY
 0000:94B4       N_KYBD_LIST
 0000:94B6       I_KEYBOARD
 0000:94B8       S_KEYBOARD
 0000:94BC       N_KYBD_VAL
 0000:94BD       N_DESIGNATES
 0000:94BF       N_CP_PRI
 0000:94C1       N_CP_SEC
 0000:94C3       N_CTY_RES
 0000:94C4       I_KYBD_ALT
 0000:94C6       S_KYBD_ALT
 0000:94CA       N_KYBD_ALT
 0000:94CB       N_KYB_LOAD
 0000:94CD       CTY_TAB_A
 0000:94CE       CTY_TAB_A_1
 0000:9582       CTY_TAB_B
 0000:9583       CTY_TAB_B_1
 0000:9628       KYBD_TAB_A
 0000:9629       KYBD_TAB_A_1
 0000:9644       KYBD_TAB_B
 0000:9645       KYBD_TAB_B_1
 0000:9660       ALT_TAB_PTR
 0000:9662       ALT_KYB_ID
 0000:9663       ALT_KYB_ID_PREV
 0000:9664       ALT_KYB_TABLE
 0000:9665       ALT_KYB_TAB_1
 0000:9674       ALT_KYBD_FR
 0000:9675       ALT_KYBD_FR_1
 0000:967B       ALT_KYBD_IT
 0000:967C       ALT_KYBD_IT_1
 0000:9682       ALT_KYBD_UK
 0000:9683       ALT_KYBD_UK_1
 0000:9689       ALT_ID_DEF
 0000:968A       S_US
 0000:968E       S_SWISS
 0000:9692       PRINTER_TABLES
 0000:9876  Abs  __acrtused
 0000:9876  Abs  __acrtmsg
 0000:99A2       N_NUMPRINT
 0000:99A4       N_PARALLEL
 0000:99A6       N_SERIAL
 0000:99A8       I_PORT
 0000:99AA       I_REDIRECT
 0000:99AC       I_PRINTER
 0000:99AE       N_PRINTER_TYPE
 0000:99AF       S_MODE_PARM
 0000:99D9       S_CP_DRIVER
 0000:99F1       S_CP_PREPARE
 0000:99FF       S_GRAPH_PARM
 0000:9A15       F_REVIEW
 0000:9A17       N_DISPLAY
 0000:9A18       N_YEAR
 0000:9A1A       N_MONTH
 0000:9A1C       N_DAY
 0000:9A1E       N_HOUR
 0000:9A20       N_MINUTE
 0000:9A22       N_SECOND
 0000:9A24       PARM_BLOCK
 0000:9A32       CMD_BUFF
 0000:9A83       S_STR40
 0000:9A85       P_STR40
 0000:9AAD       S_STR120_1
 0000:9AAF       P_STR120_1
 0000:9B27       S_STR120_2
 0000:9BA1       S_STR120_3
 0000:9C1B       S_STR120_4
 0000:9C95       SC_LINE
 0000:9D19       N_HANDLE
 0000:9D1B       N_WRITE_HANDLE
 0000:9D1D       N_WRITE_ERR_CODE
 0000:9D1F       N_RETCODE
 0000:9D21       N_COUNTER
 0000:9D23       N_WORD_1
 0000:9D25       N_WORD_2
 0000:9D27       N_WORD_3
 0000:9D29       N_WORD_4
 0000:9D2B       N_WORD_5
 0000:9D2D       N_WORD_6
 0000:9D2F       N_BYTE_1
 0000:9D30       SAVE_AREA
 0000:9D34       N_HOUSE_CLEAN
 0000:9D35       N_DSKCPY_ERR
 0000:9D36       N_DISK_1
 0000:9D38       N_DISK_2
 0000:9D3A       N_DISK_1_S1
 0000:9D3C       N_DISK_2_S1
 0000:9D3E       N_DISK_1_S2
 0000:9D40       N_DISK_2_S2
 0000:9D42       F_PARTITION
 0000:9D44       I_DESTINATION
 0000:9D46       F_FORMAT
 0000:9D48       N_DISK1_MODE
 0000:9D4A       DISK_1_TABLE
 0000:9D4B       DISK_1_VAL_ITEM
 0000:9D4C       DISK_1_START
 0000:A134       DISK_2_TABLE
 0000:A135       DISK_2_VAL_ITEM
 0000:A136       DISK_2_START
 0000:A51E       N_NAME_PART
 0000:A51F       N_SIZE_PART
 0000:A521       N_STATUS_PART
 0000:A522       N_TYPE_PART
 0000:A523       P_DRIVE_PART
 0000:A524       N_LEVEL1_PART
 0000:A525       N_LEVEL2_PART
 0000:A526       N_LEVEL3_PART
 0000:A527       N_LEVEL4_PART
 0000:A528       N_DISK_NUM
 0000:A529       STACK_INDEX
 0000:A52A       SELECT_STACK
 0000:A58E       N_DEST
 0000:A58F       INT_24_ERROR
 0000:A591       INT_24_FLAG
 0000:A592       OLD_INT_23
 0000:A596       OLD_INT_24
 0000:A59A       OLD_INT_2F
 0000:A59E       MEM_SIZE
 0000:A5A0       FORMAT_WHICH
 0000:A5A1       DISK_PANEL
 0000:A5A3       SEARCH_FILE
 0000:A5A5       SUB_ERROR
 0000:A635       HRD_BUFLEN
 0000:A637       HRD_BUFOFF
 0000:A639       HRD_BUFSEG
 0000:A6D3       INC_KS
 0000:A701       CRD_CCBVECOFF
 0000:A703       CRD_CCBVECSEG
 0000:A777       QM_OPT1
 0000:A779       QM_OPT2
 0000:A77B       QM_ID
 0000:A77D       QM_ACTIVEPAN
 0000:A7F9       PM_BASECHAR
 0000:A7FA       PM_BASEATTR
 0000:A9C8       IN_ICBID
 0000:A9D4       IN_CCBVECOFF
 0000:A9D6       IN_CCBVECSEG
 0000:A9D8       IN_CURNOR
 0000:AC32       WR_DRETLEN
 0000:AC34       WR_DRETOFF
 0000:AC36       WR_DRETSEG
 0000:AC3E       WR_HLPOPT
 0000:AC44       WR_HLPROW
 0000:AC48       WR_HCBCONT
 0000:AC85       WR_REFNUM
 0000:AC87       WR_REFOFF
 0000:AC89       WR_REFSEG
 0000:AC8B       WR_REFCNT
 0000:AC8D       WR_REFBUF
 0000:AC8F       WR_REFIELDCNT
 0000:AC91       WR_REFID
 0000:ACB9       WR_SCBID
 0000:ACBB       WR_ERROR
 0000:ACBD       WR_DATA2SEG
 0000:ACBF       WR_DATA2OFF
 0000:ACC1       WR_DATA2LEN
 0000:ACC3       WR_LVBSEG
 0000:ACC5       WR_LVBOFF
 0000:ACC7       WR_LVBLEN
 0000:ACC9       WR_LVBMEM
 0000:ACCB       WR_MAXMEMPAR
 0000:ACCF       WR_MAXHELPSZ
 0000:ACEB       WR_ICBVEC
 0000:B9B0       KD_BACKSPACE
 0000:BAC4       SOURCE_PANEL
 0000:BAC6       DEST_PANEL
 0000:BAC8       CHECK_FILE
 0000:C2D4       INSTALL
 0000:C2F1       EXIT_SELECT
 0000:C372       EXIT_SELECT2
 0000:C393       ABORT_SELECT
 0000:C4B1       $M_GET_MSG_ADDRESS
 0000:C5D8       SYSDISPMSG
 0000:CB82       $M_CLS_1
 0000:CF0F       $M_CLS_2
 0000:CF34       $M_MSGSERV_1
 0000:CF55       $M_MSGSERV_2
 0000:CF5F       INITIALIZATION
 0000:CF76       BCHAR
 0000:CF77       CHECK_VERSION
 0000:D56C       INTRO_SCREEN
 0000:D5A6       SCAN_INFO_CALL
 0000:D610       WORKSPACE_SCREEN
 0000:DDE0       DOS_LOC_SCREEN
 0000:DFDB       PRINTER_SCREEN
 0000:E430       choose_shell_screen
 0000:E7C0       DOS_PARAMETERS_SCREEN
 0000:ED60       VDISK_SCREEN
 0000:F09D       FIRST_DISK_SCREEN
 0000:F744       GET_ENTER_KEY
 0000:F760       DATE_TIME_SCREEN
 0000:FBB0       FORMAT_DISK_SCREEN
 0000:0690       CONTINUE_360
 0000:0DCD       GET_OVERLAY
 0000:0E20       DISKETTE_INSTALL
 0000:15D0       INSTALL_TO_360_DRIVE
 0000:1EA4       PROCESS_ESC_F3
 0000:1EB3       EXIT_DOS
 0000:1EC9       EXIT_DOS_CONT
 0000:1F0A       INSTALL_ERROR
 0000:1F3A       Free_Parser
 0000:1F50       CREATE_AUTOEXEC_BAT
 0000:263E       CREATE_CONFIG_SYS
 0000:2CFA       CREATE_SHELL_BAT
 0000:2DF0       GET_SCROLL_CALL
 0000:2EAE       GET_INPUT_CALL
 0000:2F3D       GET_KEY
 0000:35B6       GET_PCB
 0000:35DF       GET_SCB
 0000:3608       GET_ICB
 0000:3741       CURSOROFF
 0000:3755       CURSORON
 0000:377F       PCDISPQ_CALL
 0000:378F       PCPANEL_CALL
 0000:3803       PCMBEEP_CALL
 0000:3813       PCSLCTP_CALL
 0000:388C       PCINPUT_CALL
 0000:389F       PCGVIDO_CALL
 0000:38BF       INITIALIZE
 0000:3B6D       INSERT_DISK_ROUTINE
 0000:3BE0       MOD_XCOPY
 0000:4501       HANDLE_F3
 0000:45CF       ERROR_ACTIVE
 0000:45D0       HANDLE_ERROR_CALL
 0000:46B5       HANDLE_PANEL_CALL
 0000:46D6       HANDLE_PANEL_CALL2
 0000:46F6       HANDLE_PANEL_CALL3
 0000:46FD       HANDLE_KEYSTROKE
 0000:4710       HANDLE_CHILDREN
 0000:4750       INIT_PQUEUE_CALL
 0000:477C       PREPARE_PANEL_CALL
 0000:478E       EXEC_SCROLL_CALL
 0000:47FD       INIT_SCROLL_CALL
 0000:4859       INIT_SCROLL_W_LIST_CALL
 0000:488A       INIT_SCROLL_W_NUM_CALL
 0000:489E       SET_SCROLL_COLOUR
 0000:48A9       SET_SCROLL_CALL
 0000:4919       DISPLAY_PANEL_CALL
 0000:492F       GET_FUNCTION_CALL
 0000:4957       GET_STRING_CALL
 0000:49F0       INIT_STRING_CALL
 0000:4A60       SET_STRING_CALL
 0000:4AF1       INIT_SCROLL_STATUS_CALL
 0000:4B05       TOGGLE_SUPPORT_CALL
 0000:4B2C       UNPAD_USER_STRING
 0000:4B49       CLEAR_USER_STRING
 0000:4B5E       CHECK_MIN_MAX
 0000:4B71       CONVERT_ASCII
 0000:4BA6       CONVERT_NUMERIC
 0000:4BD7       ADD_REFRESH
 0000:4BFF       RETURN_STRING_CALL
 0000:4C2F       INIT_CHAR_CALL
 0000:4E46       GET_HELP_ID
 0000:4EFC       ADJUST_UP
 0000:4F11       ADJUST_DOWN
 0000:4F30       VIDEO_CHECK
 0000:5020       ALLOCATE_MEMORY_CALL
 0000:5068       DEALLOCATE_MEMORY_CALL
 0000:5080       ALLOCATE_HELP
 0000:50C3       DEALLOCATE_HELP
 0000:50E6       ALLOCATE_BLOCK
 0000:5125       DEALLOCATE_BLOCK
 0000:5148       ALLOCATE_LVB
 0000:5183       DEALLOCATE_LVB
 0000:5A4F       SYSPARSE
 161D:1988       INPUT
 18B2:0042       asm2cInRegs
 18B2:0050       asm2coutregs
 18B2:005E       asm2csegregs
 18B2:0084       _pinsert
 18B2:0086       _NOVAL
 18B2:008A       _format_string
 18B2:008C       _fat12_String
 18B2:0090       _fat16_String
 18B2:0094       _hilda_string
 18B2:0098       _master_boot_record
 18B2:0498       __asizds
 18B2:049A       __atopsp
 18B2:049C       __aexit_rtn
 18B2:049E       __abrktb
 18B2:04EE       __abrktbe
 18B2:04EE       __abrkp
 18B2:04F0       STKHQQ
 18B2:04F2       __acfinfo
 18B2:04FF       __aintdiv
 18B2:0503       __fac
 18B2:050B       _errno
 18B2:050D       __umaskval
 18B2:050F       __pspadr
 18B2:0511       __psp
 18B2:0513       __osversion
 18B2:0513       __osmajor
 18B2:0513       __dosvermajor
 18B2:0514       __osminor
 18B2:0514       __dosverminor
 18B2:0515       __osmode
 18B2:0516       __oserr
 18B2:0516       __doserrno
 18B2:0518       __nfile
 18B2:051A       __osfile
 18B2:052E       ___argc
 18B2:0530       ___argv
 18B2:0532       _environ
 18B2:0534       __pgmptr
 18B2:053A       __child
 18B2:053C       __ovlflag
 18B2:053D       __intno
 18B2:053E       __ovlvec
 18B2:0542       __adbgmsg
 18B2:055C       __fpinit
 18B2:0642       _edata
 18B2:0650       _reboot_flag
 18B2:0651       _dx_buff
 18B2:066C       _OneDiskStatusEntry
 18B2:0676       _video_mode
 18B2:0678       _max_head
 18B2:067A       _input_col
 18B2:067C       _total_mbytes
 18B2:0680       _input_data
 18B2:0682       _regs
 18B2:0690       _primary_flag
 18B2:0691       _next_letter
 18B2:0692       _display_page
 18B2:0694       _input_row
 18B2:0696       _good_disk
 18B2:0698       _ext_table
 18B2:0BA8       _segregs
 18B2:0BB0       _extended_buff
 18B2:0BB2       _total_disk
 18B2:0BB6       _primary_buff
 18B2:0BB8       _logical_flag
 18B2:0BB9       _number_of_drives
 18B2:0BBA       _extended_flag
 18B2:0BBC       _sort
 18B2:0BD4       _no_fatal_error
 18B2:0BD5       _cur_disk_buff
 18B2:0BD6       _insert
 18B2:0EF6       _part_table
 18B2:0FCE       _max_sector
 18B2:0FD0       _boot_record
 18B2:11D0       _logical_buff
 18B2:11D2       _cur_disk
 18B2:11D3       _valid_input
 18B2:11D4       _free_space
 18B2:1294       _required_cyls
 18B2:1298       _errorlevel
 18B2:1299       _max_partition_size
 18B2:12A0       _end

Program entry point at 0C2D:0004
